Subject: [ippm] Retrasmitted packets...

From: Claus Rugani Topke <[email-masked]>
Date: Wed, 7 Mar 2001 09:16:26 -0300

Hi,

I'm not sure what should be considered as "retransmited packet" or
"retransmitted data" in a TCP flow...

I fould the following flow in tcpdump output:
982027803.529734 222.222.222.194.1094 > 333.333.333.2.80: . 7885497:7885497(0) ack 1439554681 win 32120 (DF) (ttl 122, id 42242)
982027803.542848 222.222.222.194.1094 > 333.333.333.2.80: . 7885497:7885497(0) ack 1439555705 win 32120 (DF) (ttl 122, id 42498)
982027803.556465 222.222.222.194.1094 > 333.333.333.2.80: . 7885497:7885497(0) ack 1439556596 win 32120 (DF) (ttl 122, id 42754)
982027803.647738 222.222.222.194.1094 > 333.333.333.2.80: . 7885497:7885497(0) ack 1439556596 win 32120 (DF) (ttl 122, id 43522)

These packets where retransmissions ?

Is there any place where I can found a good definition about flow retransmissions ?

Thanks in advance,
Claus
_______________________________________________
ippm mailing list
[email-masked]
http://mailhost.advanced.org/mailman/listinfo/ippm